:020000040000FA
:060000000DEF0AF01200F2
:02002A000000D4
:04002C00800EE66EEE
:1000300022DAE552430E706E7168070E726E100E72
:10004000736E606A0F01506B240E006F600E016FBB
:10005000240E046F200E056F086B096B0C6B0D6B83
:10006000106B116B146B156B186B600E196F1C6B9A
:100070001D6BE66A00DAE5521200D9CFE6FFE1CF48
:10008000D9FF190EE126D950060FE96EDACFEAFF43
:10009000400EEE6E0F0EED6ED950080FE96EDACFFE
:1000A000EAFF300EEE6E0F0EED6ED9500A0FE96EBC
:1000B000DACFEAFF200EEE6E0F0EED6EDF6A020E53
:1000C000DF5C01E3D1D0D950060F0B6EDACF0CF014
:1000D000DF50020D0B50F324E96E0C50F420EA6E51
:1000E000020EEECFDBFF030EEDCFDBFF020EDBCF08
:1000F00006F0030EDBCF07F0040E06C0DBFF050E93
:1001000007C0DBFF020EDBCFE9FF030EDBCFEAFF08
:10011000EF50080B01E0A6D0FC0E0B6E020EDBCFF9
:10012000E9FF030EDBCFEAFF0B50EF16F70EDB50B3
:10013000030B0B6E020EDBCFE9FF030EDBCFEAFFF2
:100140000B50EF12F70EDBAC08D0F80EDB50400975
:10015000E76E180EE7CFDBFF06D0F80EDB50E76E38
:10016000180EE7CFDBFF050EE76E020EDBCFE9FFCF
:10017000030EDBCFEAFFE750E926000EEA22180E55
:10018000DBCFEFFFF70EDBAA06D0010EF36E180EE1
:10019000F3CFDBFF02D0180EDB6ADBCFE6FFD950CE
:1001A000FB0FE96EFF0EDA20EA6EEECFE6FFEECF30
:1001B000E6FFEECFE6FFEFCFE6FF010EE76E020EA1
:1001C000DBCF0BF0030EDBCF0CF0E7500B26000E5D
:1001D0000C220BC0E6FF0CC0E6FF62D9F56E070EDD
:1001E000E15EF550D950020FE96EDACFEAFF060E54
:1001F000EE26000EED22010EDB6AF80EDB50F36EE8
:10020000010EDBCFF4FFF350F45C1AE2F90EDBCF02
:10021000E9FFDB2AFA0EDBCFEAFF01E3DB2AEF502E
:10022000E66E020EDBCFE9FFDB2A030EDBCFEAFF2F
:1002300001E3DB2AE552E750EF6E010EDB2ADDD742
:10024000040EDBCFE9FF050EDBCFEAFFEF50040B16
:1002500007E1040EDBCFE9FF050EDBCFEAFFEF86F7
:10026000010E04D0DF2A2BD7000E00D0D9CFE1FF3A
:10027000E552E7CFD9FF1200D9CFE6FFE1CFD9FF92
:10028000060EE12600016D6B60AE15D0A49074AE31
:1002900008D0F70EDBCFE9FFF80EDBCFEAFFEF86E1
:1002A000749E6D916050010B01E06D81600EDE6EF9
:1002B0000F0EDD6E23D00F0150AF1ED0A49274AC90
:1002C00008D0F70EDBCFE9FFF80EDBCFEAFFEF86B1
:1002D000749C070E501500016D6F020E6D5D07E2F4
:1002E000F70EDBCFE9FFF80EDBCFEAFFEF8E500E03
:1002F000DE6E0F0EDD6E02D0000EB7D0D9CFE9FF53
:10030000DACFEAFF020EEECFDBFF030EEDCFDBFF0D
:10031000F70EDBCFE9FFF80EDBCFEAFFEF6ADECFA7
:10032000E9FFDDCFEAFF050EE926000EEA22050E01
:10033000EFCFDBFFDB500F0BE66EF90EDBCFE9FFF3
:10034000FA0EDBCFEAFFE552E750EF6ED950050F0A
:10035000E96EDACFEAFFEF50400B08E000D0F70E6D
:10036000DBCFE9FFF80EDBCFEAFFEF8CDECFE9FF52
:10037000DDCFEAFF020EE926000EEA22050EEFCFDE
:10038000DBFFD950050FE96EDACFEAFFEF50080B1B
:100390000DE0F70EDBCFE9FFF80EDBCFEAFFEF8AC7
:1003A000010EF36E050EF3CFDBFF02D0050EDB6A04
:1003B000DBCFE6FFFD0EDBCFE6FFFE0EDBCFE6FF79
:1003C000DECF0BF0DDCF0CF0010E0B26000E0C2261
:1003D0000BC0E6FF0CC0E6FF3FD9F56E050EE15EEF
:1003E000F550060EDE26000EDD22F90EDBCFE9FF0A
:1003F000FA0EDBCFEAFF050EEFCFDBFF040EDB6A60
:10040000050EDB50F36E040EDBCFF4FFF350F45C0B
:1004100019E2DFCFE9FFDF2A010EDBCFEAFF01E3BC
:10042000DB2AEF50E66EFB0EDBCFE9FFDB2AFC0E8A
:10043000DBCFEAFF01E3DB2AE552E750EF6E040E63
:10044000DB2ADED7A4AE08D0F70EDBCFE9FFF80E2B
:10045000DBCFEAFFEF88A49E020EDBCFE9FF030E9D
:10046000DBCFEAFFEF9E010E00D0D9CFE1FFE552CE
:10047000E7CFD9FF1200D9CFE6FFE1CFD9FF1F0E9A
:100480006F16FE0EDB506F12E00E6E140B6EFE0E3A
:10049000DB500B5C01E0F8D7E552E7CFD9FF120043
:1004A000D9CFE6FFE1CFD9FF020EE126D950F90FEF
:1004B0000B6EFF0EDA200C6E0BC0DEFF0CC0DDFFF2
:1004C000F80EDB503BE1DECFE9FFDDCFEAFFEF5076
:1004D000E840E840E8401F0BE66EFD0EDBCFE9FF89
:1004E000FE0EDBCFEAFFE552E750EF6EDECFE9FF0D
:1004F000DDCFEAFFEE52EF50200DF3CF0BF0FD0EF3
:10050000DBCFE9FFFE0EDBCFEAFF0B50EF12FD0E53
:10051000DB2AFE0E01E3DB2ADECFE9FFDDCFEAFFB7
:10052000EF50200DF350E66EFD0EDBCFE9FFFE0E1F
:10053000DBCFEAFFE552E750EF6E88D0DECFE9FF70
:10054000DDCFEAFF020EE926000EEA22EF50E00BB3
:10055000E838E840E66EFD0EDBCFE9FFFE0EDBCFAC
:10056000EAFFE552E750EF6EDECFE9FFDDCFEAFFAD
:10057000030EE926000EEA22EF50080DF3CF0BF030
:10058000FD0EDBCFE9FFFE0EDBCFEAFF0B50EF12D3
:10059000FD0EDB2AFE0E01E3DB2ADECFE9FFDDCF15
:1005A000EAFF020EE926000EEA22EF50080DF35092
:1005B000E00BE66EFD0EDBCFE9FFFE0EDBCFEAFFC0
:1005C000E552E750EF6EFD0EDBCFE9FFFE0EDBCF0D
:1005D000EAFFEF86DECFE9FFDDCFEAFF020EE92674
:1005E000000EEA22EF50030B0B6EFD0EDBCFE9FF8E
:1005F000FE0EDBCFEAFF0B50EF12FD0EDB2AFE0EE4
:1006000001E3DB2ADECFE9FFDDCFEAFFEE52EF5058
:10061000E66EFD0EDBCFE9FFFE0EDBCFEAFFE55213
:10062000E750EF6EFD0EDB2AFE0E01E3DB2ADECF84
:10063000E9FFDDCFEAFFEF50E66EFD0EDBCFE9FF0D
:10064000FE0EDBCFEAFFE552E750EF6ED9CFE1FFB8
:10065000E552E7CFD9FF1200D9CFE6FFE1CFD9FFAE
:10066000020EE126FB0EDBCFDEFFDBCFDDFFFA0E55
:10067000DB504DE1FD0EDBCFE9FFFE0EDBCFEAFFE5
:10068000EF50080DF350E66EDECFE9FFDDCFEAFF55
:10069000E552E750EF6EFD0EDBCFE9FFFE0EDBCF3C
:1006A000EAFFEF50E00BE838E840E66EDECFE9FF06
:1006B000DDCFEAFFEE52E552E750EF6EFD0EDB2A8A
:1006C000FE0E01E3DB2AFD0EDBCFE9FFFE0EDBCFE2
:1006D000EAFFEF50E00BE838E8400B6EDECFE9FFB1
:1006E000DDCFEAFF0B50EF12DECFE9FFDDCFEAFFEF
:1006F000020EE926000EEA22EF6ADECFE9FFDDCF27
:10070000EAFF030EE926000EEA22EF6A84D0FD0E0E
:10071000DBCFE9FFFE0EDBCFEAFFEF50200DF350F9
:10072000E66EDECFE9FFDDCFEAFF020EE926000E1E
:10073000EA22E552E750EF6EFD0EDBCFE9FFFE0E39
:10074000DBCFEAFFEF50E840E840E8401F0BE66EE1
:10075000DECFE9FFDDCFEAFF030EE926000EEA2235
:10076000E552E750EF6EFD0EDB2AFE0E01E3DB2AB9
:10077000FD0EDBCFE9FFFE0EDBCFEAFFEF50030BF0
:100780000B6EDECFE9FFDDCFEAFF020EE926000E99
:10079000EA220B50EF12FD0EDBCFE9FFFE0EDBCF9E
:1007A000EAFFEF50E00BE840E840E8401F0B0B6E1B
:1007B000DECFE9FFDDCFEAFF020EE926000EEA22D6
:1007C0000B50EF12FD0EDB2AFE0E01E3DB2AFD0EBD
:1007D000DBCFE9FFFE0EDBCFEAFFEF50E66EDECFA8
:1007E000E9FFDDCFEAFFEE52E552E750EF6EFD0E76
:1007F000DB2AFE0E01E3DB2AFD0EDBCFE9FFFE0E56
:10080000DBCFEAFFEF50E66EDECFE9FFDDCFEAFF98
:10081000E552E750EF6ED9CFE1FFE552E7CFD9FFC0
:020820001200C4
:0E082200D9CFE6FFE1CFD9FF070EE126C16E68
:10083000C26AB46E926A2B0E936E800E946E080E8E
:10084000956E966A829082828294400EE66EE66A87
:100850003C0EE66E79EC09F0E552E552E552420EA7
:100860000B6E120E0C6E0D6A0BC0E6FF0CC0E6FF9D
:100870000DC0E6FFADEC09F0E552E552E5521F0E62
:100880000B6E120E0C6E0D6A0BC0E6FF0CC0E6FF7D
:100890000DC0E6FFADEC09F0E552E552E552060E5B
:1008A0000B6E120E0C6E0D6A0BC0E6FF0CC0E6FF5D
:1008B0000DC0E6FFADEC09F0E552E552E552DF0E62
:1008C0000B6E110E0C6E0D6A0BC0E6FF0CC0E6FF3E
:1008D0000DC0E6FFADEC09F0E552E552E552D9EC6A
:1008E00007F000095CE0D10E0B6E110E0C6E0D6A64
:1008F0000BC0E6FF0CC0E6FF0DC0E6FFADEC09F053
:10090000E552E552E552B80E0B6E110E0C6E0D6AF3
:100910000BC0E6FF0CC0E6FF0DC0E6FFADEC09F032
:10092000E552E552E552010EF36E030EF3CFDBFF05
:10093000DB50030833E3D9EC07F0CC0EE66EFCEC99
:1009400007F0E552440EE66EFCEC07F0E55281EC50
:1009500008F0000901E0FBD7D9EC07F0CC0EE66EF9
:10096000FCEC07F0E552BE0EE66EFCEC07F0E5523B
:10097000010EF36E020EF3CFDBFFDB50090806E336
:1009800039EC08F0DF6E020EDB2AF7D7880EE66E30
:10099000DFEC09F0E552030EDB2ACAD710D0A70E10
:1009A0000B6E110E0C6E0D6A0BC0E6FF0CC0E6FF5D
:1009B0000DC0E6FFADEC09F0E552E552E5520B0E35
:1009C000E66E1DEC06F0E552000EE66EE66AA00E3D
:1009D000E66E95EC06F0E552E552E55200092BE192
:1009E0009A0E0B6E110E0C6E0D6A0BC0E6FF0CC05A
:1009F000E6FF0DC0E6FFADEC09F0E552E552E55229
:100A00001CEC07F000016B6F1CEC07F000016A6F33
:100A100026EC07F08B0E0B6E110E0C6E0D6A0BC0E0
:100A2000E6FF0CC0E6FF0DC0E6FFADEC09F0E552B5
:100A3000E552E55210D07B0E0B6E110E0C6E0D6A56
:100A40000BC0E6FF0CC0E6FF0DC0E6FFADEC09F001
:100A5000E552E552E55216EC00F0710E0B6E110EE8
:100A60000C6E0D6A0BC0E6FF0CC0E6FF0DC0E6FF82
:100A7000ADEC09F0E552E552E552530E0B6E110E46
:100A80000C6E0D6A0BC0E6FF0CC0E6FF0DC0E6FF62
:100A9000ADEC09F0E552E552E552829281B0FED705
:100AA0008284D9EC07F0CC0EE66EFCEC07F0E55240
:100AB000440EE66EFCEC07F0E55281EC08F000090C
:100AC00001E0FBD7D9EC07F0CC0EE66EFCEC07F0AA
:100AD000E552BE0EE66EFCEC07F0E55239EC08F08C
:100AE000DF6E39EC08F0E76E010EE7CFDBFFF36E47
:100AF000020EF3CFDBFFDB50070809E339EC08F007
:100B0000E76E030EE7CFDBFF020EDB2AF4D7040EFD
:100B1000DB6A010EDB50070841E3010EDB50E66E95
:100B2000D950050FE96EDACFEAFFE552E750EE6ED5
:100B3000ED6A050EDBCF0BF0060EDBCF0CF00BC021
:100B40000CF00B6A050E0BC0DBFF060E0CC0DBFFC2
:100B5000DF50E76E050EDBCF0BF0060EDBCF0CF09F
:100B6000E7500B26000E0C22050E0BC0DBFF060E15
:100B70000CC0DBFF050EDBCF0BF0060EDBCF0CF05D
:100B800000010B506A5D0C506B5906E2010EF36ECA
:100B9000040EF3CFDBFF02D0040EDB6A040EDB5041
:100BA00017E0E66A020EE66ED9CFE6FFDACFE6FF7F
:100BB000230EE66E010EE66EE66AE66A3DEC00F094
:100BC000F56E080EE15EF550000901E1EAD716D096
:100BD000E66A020EE66ED9CFE6FFDACFE6FF210E17
:100BE000E66E010EE66EE66AE66A3DEC00F0F56E32
:100BF000080EE15EF550000901E1EAD74A0E0B6EDE
:100C0000110E0C6E0D6A0BC0E6FF0CC0E6FF0DC0A6
:100C1000E6FFADEC09F0E552E552E55281A0FED7C2
:100C2000500EE66EDFEC09F0E552829437D7D9CF4B
:0A0C3000E1FFE552E7CFD9FF120003
:060C3A00D9CFE6FFE1CF77
:100C4000D9FF3F0EC716C66AC56AC68694869488C1
:100C5000C68AFE0EDB50C86EE552E7CFD9FF120000
:100C6000D9CFE6FFE1CFD9FF020EE126FC0EDBCFA4
:100C7000DEFFDBCFDDFFC750040B01E0010E0B6E82
:100C80001F0EC5140B1001E0F6D7C580C5B0FED706
:100C9000A1A602D0010E43D0FE0EDBCFE6FF6FD936
:100CA000E552000902E0010E3AD0C750040B01E002
:100CB000010E0B6E1F0EC5140B1001E0F6D7C5BC5C
:100CC0002CD0010EDBCFE6FF5AD9E552000902E035
:100CD000010E25D0C750040B01E0010E0B6E1F0E54
:100CE000C5140B1001E0F6D7DFCFE6FF48D9E55277
:100CF000000902E0010E13D0C750040B01E0010E01
:100D00000B6E1F0EC5140B1001E0F6D7C5BC03D047
:100D1000000E05D004D0020E02D0020E00D0D9CFB2
:100D2000E1FFE552E7CFD9FF1200D9CFE6FFE1CFCF
:100D3000D9FFE652FC0EDBCFE6FFFD0EDBCFE6FF70
:100D4000FE0EDBCFE6FF8CDFE552E552E552DF6EAB
:100D5000DF5002E0DF5030D0BCD8DF6EDF5002E061
:100D6000DF502AD0C750040B01E0010E0B6E1F0E9E
:100D7000C5140B1001E0F6D7C580C5B0FED7A1A6FB
:100D800002D0010E19D0FE0EDB28E66EF8D8E5522F
:100D9000000902E0010E10D0C750040B01E0010E63
:100DA0000B6E1F0EC5140B1001E0F6D7C5BC02D0A8
:100DB000000E02D0020E00D0E552E552E7CFD9FF77
:100DC0001200D9CFE6FFE1CFD9FFC750040B01E0F5
:100DD000010E0B6E1F0EC5140B1001E0F6D7FE0EB0
:100DE000DBCFE6FFCCD8E552000902E0010E10D0BF
:100DF000C750040B01E0010E0B6E1F0EC5140B1043
:100E000001E0F6D7C5BC02D0000E02D0020E00D021
:100E1000E552E7CFD9FF1200C750040B01E0010EE5
:100E20000B6E1F0EC5140B1001E0F6D7C584C5B4B8
:100E3000FED7000E00D01200B6D8C5B6FED7C59AB0
:100E4000C588C5B8FED7C95000D01200ACD8C5B609
:100E5000FED7C58AC588C5B8FED7C584C5B4FED738
:100E6000000E00D01200D9CFE6FFE1CFD9FFE65245
:100E7000FC0EDBCFE6FFFD0EDBCFE6FFFE0EDBCF89
:100E8000E6FF53DFE552E552E552DF6EDF5002E048
:100E9000DF501AD0F90EDBCFF3FFDB06F350000969
:100EA0000FE0CADFE66EFA0EDBCFE9FFDB2AFB0EAE
:100EB000DBCFEAFF01E3DB2AE552E750EF6EEAD72A
:100EC000C5DFDF6EDF5000D0E552E552E7CFD9FF36
:100ED0001200C750040B01E0010E0B6E1F0EC5146B
:100EE0000B1001E0F6D7C584C5B4FED7A1A602D089
:100EF000010E02D0000E00D01200D9CFE6FFE1CFE4
:100F0000D9FFE652C750040B01E0010E0B6E1F0E15
:100F1000C5140B1001E0F6D7C580C5B0FED7A1A659
:100F200003D0010E27D01DD0FE0EDBCFE6FF27D861
:100F3000E552000902E0010E1DD0C750040B01E08C
:100F4000010E0B6E1F0EC5140B1001E0F6D7A1A603
:100F500002D0010E0FD0C5BC02D0DF6A02D0040E51
:100F6000DF6EC584C5B4FED7A1A602D0010E02D0A3
:100F7000DF5000D0E552E552E7CFD9FF1200D9CFBC
:100F8000E6FFE1CFD9FFFE0EDB50C96EC6AE03D03F
:100F9000FF0E05D004D0C7B0FED7000E00D0E5523A
:100FA000E7CFD9FF1200C586C7A0FED7C95000D031
:020FB00012002D
:0E0FB200D9CFE6FFE1CFD9FFE652DF6A939A6E
:100FC000819AF00EE66E19EC0AF0E552938A280E2B
:100FD000E66E19EC0AF0E55281BA02D0010EDF6E1E
:100FE000C80EE66E19EC0AF0E552DF5000D0E5526B
:100FF000E552E7CFD9FF1200D9CFE6FFE1CFD9FF05
:10100000E652DF6A080EDF5C2FE2FE0EDB50DF5295
:1010100006E0DFCFF3FFE8327F0BF306FCE1010BC4
:1010200014E0939A819A030EE66E19EC0AF0E552E9
:10103000938A250EE66E19EC0AF0E552938A010EAA
:10104000E66E19EC0AF0E5520DD0939A819A280EBB
:10105000E66E19EC0AF0E552938A010EE66E19EC81
:101060000AF0E552DF2ACED7E552E552E7CFD9FFA5
:101070001200D9CFE6FFE1CFD9FF030EE126010E22
:10108000DB6A020EDB6ADF6A080EDF5C31E2819AFE
:10109000939A020EE66E19EC0AF0E552938A020E5C
:1010A000E66E19EC0AF0E5528150200B01E0010ECA
:1010B000E76E010EE7CFDBFFD950010FE96EDACF03
:1010C000EAFFDF50070B04E0EF46EF90E806FCE193
:1010D000020EDBCFE7FF010EDB50E712020EE7CF77
:1010E000DBFF240EE66E19EC0AF0E552DF2ACCD7BE
:1010F000020EDB5000D0D9CFE1FFE552E7CFD9FF98
:101100001200D9CFE6FFE1CFD9FFE652DF6A819A1C
:10111000939A020EE66E19EC0AF0E552938A020EDB
:10112000E66E19EC0AF0E5528150200B01E0010E49
:10113000DF6E240EE66E19EC0AF0E552DF5000D0A7
:0A114000E552E552E7CFD9FF120097
:06114A005458204D5347EC
:101150000A0D005072656D6572652053573020701E
:101160006572206F676E6920696E76696F2E0A0D51
:101170000043414E204F4B200A0D00454550524F31
:101180004D204E4F2D4F4B200A0D0054454D502EF3
:101190004D4158204F4B200A0D00454550524F4DB0
:1011A000204F4B200A0D0044533138423230204E3C
:1011B0004F2D4F4B200A0D00496E697A69616C69A9
:1011C0007A7A6120445331384232302E2E2E0A0D65
:1011D0000044533138423230204F4B200A0D002D4D
:1011E0002D2D2D2D2D2D2D2D2D2D2D2D2D2D2D2D2F
:1011F0002D2D2D2D2D2D2D2D2D2D2D2D2D2D2D2D1F
:101200002D2D2D0A0D004175746F72653A204361D2
:10121000726C6F205461757261736F200A0D004605
:1012200069726D7761726520766572312E30202D7E
:1012300020436F72736F2043414E2D425553200A55
:101240000D00417676696F204E4F444F2043414E4A
:04125000200A0D0063
:0C1254002A0EF66E000EF76E000EF86E0B
:1012600000010900F550656F0900F550666F03E154
:10127000656701D03DD00900F550606F0900F55059
:10128000616F0900F550626F09000900F550E96EC1
:101290000900F550EA6E090009000900F550636F76
:1012A0000900F550646F09000900F6CF67F0F7CF29
:1012B00068F0F8CF69F060C0F6FF61C0F7FF62C068
:1012C000F8FF0001635302E1645307E00900F550A1
:1012D000EE6E6307F8E26407F9D767C0F6FF68C0EF
:1012E000F7FF69C0F8FF00016507000E665BBFD716
:0212F0001200EA
:0E12F200D9CFE6FFDACFE6FFE1CFD9FFE2CF9A
:10130000DAFFAC6AAB6AFD0EDBB0AC88DBA202D0C0
:10131000AC8CAB8CDBB4AC8EDBA602D0AB8801D03E
:10132000AB8ADBA802D0AC8401D0AC949E98DBAC35
:1013300002D09D8A01D09D9A9E9ADBAE02D09D88F4
:1013400001D09D98FB0EDB50AF6EAC8AAB8EE552A0
:0A135000E5CFDAFFE7CFD9FF120066
:06135A00D9CFE6FFDACF57
:10136000E6FFE1CFD9FFE2CFDAFFACA2FED7FB0E5A
:10137000DBCFF6FFFC0EDBCFF7FFFD0EDBCFF8FF78
:101380000800F550E66EF6EC09F0E552D950FB0F77
:10139000E96EFF0EDA20EA6EEFCFF6FFEE2AEFCF0E
:1013A000F7FF000EEE22EFCFF8FFEE220800F55017
:0E13B000DCE1E552E5CFDAFFE7CFD9FF12000E
:0213BE00FF0E20
:1013C000E3500F6EEF0E01D0F30EE76EE72EE6EF5F
:1013D00009F00C0E0E6EE76AE72EECEF09F00E2E08
:0C13E000EBEF09F00F2EE4EF09F0120013
:0413EC00D9CFE6FF70
:1013F000DACFE6FFE1CFD9FFE2CFDAFFACAC04D021
:10140000AC9000016CB3AC80FD0EDB50AD6EE552CC
:0A141000E5CFDAFFE7CFD9FF1200A5
:06141A0015EE00F025EEC6
:1014200000F0F86A0A9C2AEC09F011EC04F0FDD7F0
:021430001200A8
:0E143200FF0EE350E84E1200000000D000D084
:0814400000D0E82EFAD71200DB
:020000040030CA
:08000000FFFAFFFEFFFFFBFF0A
:00000001FF
